:100000000C9462000C948A000C948A000C948A0070
:100010000C948A000C948A000C948A000C948A0038
:100020000C948A000C948A000C948A000C948A0028
:100030000C948A000C948A000C948A000C948A0018
:100040000C9453020C948A000C94C3020C949D02ED
:100050000C948A000C948A000C948A000C948A00F8
:100060000C948A000C948A000000000023002600F3
:10007000290000000008000201000003040700003E
:1000800000000000000000000000250028002B00F8
:1000900000000000240027002A00040404040404D3
:1000A0000404020202020202030303030303010227
:1000B00004081020408001020408102001020408F6
:1000C00010201C0811241FBECFEFD8E0DEBFCDBF2B
:1000D00011E0A0E0B1E0E0EFF0E102C005900D9288
:1000E000A23AB107D9F722E0A2EAB1E001C01D921D
:1000F000A838B207E1F710E0C2E6D0E004C02197CB
:10010000FE010E945108C136D107C9F70E94F502CD
:100110000C9476080C94000090E0FC01E255FF4F2F
:100120002491FC01E656FF4F8491882399F090E0DA
:10013000880F991FFC01E057FF4FA591B491FC0176
:10014000EA57FF4F859194918FB7F894EC91E22B89
:10015000EC938FBF0895833081F028F4813099F0BB
:100160008230A1F008958730A9F08830B9F084304A
:10017000D1F4809180008F7D03C0809180008F77C3
:1001800080938000089584B58F7702C084B58F7DF9
:1001900084BD08958091B0008F7703C08091B00036
:1001A0008F7D8093B0000895CF93DF93282F30E0A8
:1001B000F901EE58FF4F8491F901E255FF4FD491B8
:1001C000F901E656FF4FC491CC2391F081110E94B2
:1001D000AB00EC2FF0E0EE0FFF1FE859FF4FA591A9
:1001E000B491EC91ED2381E090E021F480E002C035
:1001F00080E090E0DF91CF9108951F93CF93DF933C
:10020000282F30E0F901EE58FF4F8491F901E255B3
:10021000FF4FD491F901E656FF4FC491CC23C9F0AA
:10022000162F81110E94AB00EC2FF0E0EE0FFF1FA4
:10023000EA57FF4FA591B4918FB7F894111105C0FB
:100240009C91ED2FE095E92302C0EC91ED2BEC930E
:100250008FBFDF91CF911F9108958230910538F0C3
:10026000880F991F880F991F05970197F1F7089537
:10027000CF92DF92EF92FF920F931F93CF93DF9372
:100280006C017A018B01C0E0D0E0CE15DF0589F06A
:10029000D8016D918D01D601ED91FC910190F08115
:1002A000E02DC6010995892B11F47E0102C021962B
:1002B000ECCFC701DF91CF911F910F91FF90EF908D
:1002C000DF90CF900895FC01918D828D981761F099
:1002D000828DDF01A80FB11D5D968C91928D9F5F7D
:1002E0009F73928F90E008958FEF9FEF0895FC0128
:1002F000918D828D981731F0828DE80FF11D858DDB
:1003000090E008958FEF9FEF0895FC01918D228D6D
:10031000892F90E0805C9F4F821B91098F739927F2
:1003200008958BEE91E00E94850121E0892B09F46C
:1003300020E0822F0895FC01848DDF01A80FB11DFC
:10034000A35ABF4F2C91848D90E001968F7399270B
:10035000848FA689B7892C93A089B1898C918064F8
:100360008C93938D848D981306C00288F389E02DB9
:1003700080818F7D80830895EF92FF920F931F936A
:10038000CF93DF93EC0181E0888F9B8D8C8D981348
:1003900005C0E889F989808185FD24C0F62E0B8D82
:1003A00010E00F5F1F4F0F731127E02E8C8DE812A6
:1003B0000CC00FB607FCFACFE889F989808185FF68
:1003C000F5CFCE010E949B01F1CF8B8DFE01E80F8E
:1003D000F11DE35AFF4FF0820B8FEA89FB89808180
:1003E000806207C0EE89FF896083E889F98980818E
:1003F0008064808381E090E0DF91CF911F910F9125
:10040000FF90EF900895CF93DF93EC01888D8823C0
:10041000C9F0EA89FB89808185FD05C0A889B98971
:100420008C9186FD0FC00FB607FCF5CF808185FF4C
:10043000F2CFA889B9898C9185FFEDCFCE010E94BA
:100440009B01E7CFDF91CF91089580E090E0892B69
:1004500029F00E94910181110C9400000895CF931E
:10046000DF93009779F0FC0101900020E9F73197C4
:10047000AF01481B590BBC018BEE91E00E94380183
:10048000EC0102C0C0E0D0E042E050E060E171E089
:100490008BEE91E00E9438018C0F9D1FDF91CF9170
:1004A00008950E9471081F920F920FB60F921124A7
:1004B0002F933F938F939F93AF93BF938091E701C7
:1004C0009091E801A091E901B091EA013091E60133
:1004D00023E0230F2D3720F40196A11DB11D05C087
:1004E00026E8230F0296A11DB11D2093E6018093FB
:1004F000E7019093E801A093E901B093EA018091AC
:10050000E2019091E301A091E401B091E50101962F
:10051000A11DB11D8093E2019093E301A093E4013A
:10052000B093E501BF91AF919F918F913F912F9132
:100530000F900FBE0F901F9018951F920F920FB63D
:100540000F9211242F933F934F935F936F937F9359
:100550008F939F93AF93BF93EF93FF938BEE91E0B5
:100560000E949B01FF91EF91BF91AF919F918F915D
:100570007F916F915F914F913F912F910F900FBE9F
:100580000F901F9018951F920F920FB60F92112483
:100590002F938F939F93EF93FF93E091FB01F09143
:1005A000FC018081E0910102F091020282FD12C003
:1005B0009081809104028F5F8F73209105028217D2
:1005C00051F0E0910402F0E0E551FE4F958F8093E9
:1005D000040201C08081FF91EF919F918F912F9133
:1005E0000F900FBE0F901F901895CF93DF9300D000
:1005F00000D0CDB7DEB7789484B5826084BD84B571
:10060000816084BD85B5826085BD85B5816085BD0D
:1006100080916E00816080936E00109281008091C5
:10062000810082608093810080918100816080934D
:100630008100809180008160809380008091B10072
:1006400084608093B1008091B00081608093B0009D
:1006500080917A00846080937A0080917A00826031
:1006600080937A0080917A00816080937A008091F3
:100670007A00806880937A001092C1008DE00E9419
:100680008C0061E088E00E94FD0061E083E00E9450
:10069000FD00E091FB01F091FC0182E08083E0919C
:1006A000F701F091F8011082E091F901F091FA015F
:1006B0008FEC808310920302E091FF01F091000221
:1006C00086E08083E091FD01F091FE0180818061F0
:1006D0008083E091FD01F091FE018081886080833C
:1006E000E091FD01F091FE01808180688083E091BE
:1006F000FD01F091FE0180818F7D80838BE193E08D
:100700000197F1F77AE0772EE4E66E2EFBE88F2E64
:10071000992493948BEE91E00E9485011816190696
:100720009CF58BEE91E00E9485011816190664F580
:100730008BEE91E00E9463019091A3019923F9F05F
:10074000E091A2018E3379F0AE2FB0E0AC53BE4FF2
:100750008C93EF5FED3118F4E093A20115C02CE10A
:100760002093A20111C0F0E0EC53FE4F10821092D2
:10077000A3011092A20141E04093E10105C08C3336
:1007800019F451E05093A3018091E101882309F409
:1007900050C41092E1018091C401843569F483E171
:1007A00091E00E942F0283E391E00E942F0261E01A
:1007B00084E00E94FD003DC48D3409F038C1809171
:1007C000C901082E000C990BC097789E9001799E64
:1007D000300D11240091CA01002E000C110B0053A2
:1007E0001109020F131F2091CC01022E000C330BB4
:1007F00020533109729EC001739E900D11242091E7
:10080000CD01022E000C330B20533109F901E80F02
:10081000F91FFC83EB835090CF018091D101082E0A
:10082000000C990BC097689E7001699EF00C112412
:100830008091D201082E000C990BC097789E9001F0
:10084000799E300D11242E0D3F1DE090D3010E2C0A
:10085000000CFF08C701C0977901E80EF91EA091AE
:10086000D5010A2E000CBB0BD09720E836E948E9E9
:1008700050E00E9449085B016C01A091D6010A2E4C
:10088000000CBB0BD09720E432E44FE050E00E9414
:100890004908A60EB71EC81ED91EA091D7010A2E60
:1008A000000CBB0BD09720EA36E841E050E00E94F4
:1008B0004908A60EB71EC81ED91EA091D8010A2E3F
:1008C000000CBB0BD09740E157E2A49FF001A59F1D
:1008D000F00DB49FF00D1124AF01FF0F660B770BE5
:1008E000A40EB51EC61ED71EA091D9010A2E000C5B
:1008F000BB0BD09788EE93E0A89FA001A99F500D55
:10090000B89F500D1124052E000C660B770B4A0D75
:100910005B1D6C1D7D1DE091DA01AE2FEE0FBB0B50
:10092000FD01F0976E9E90016F9E300D1124C9015C
:10093000330FAA0BBB0B5A016B01A80EB91ECA1EBE
:10094000DB1E4091DB01A42F440FBB0BAD014053D4
:100950005109749EC001759E900D1124092E000C42
:10096000AA0BBB0BB601A501480F591F6A1F7B1FBD
:10097000A091DC010A2E000CBB0BD097CD01BB0F60
:10098000AA0BBB0B5A016B01A80EB91ECA1EDB1EB7
:100990008091C601082E000C990BC097789E90019B
:1009A000799E300D11248091C701082E000C990BFF
:1009B000C097820F931F89830E948C00802F0E9412
:1009C0008C008B810E948C0090E3591202C060E081
:1009D00001C061E0802F0E94FD0060E08B810E94D9
:1009E000FD00212C312C2101239461E0A214B304D9
:1009F000C404D5049CF089810E94FD00C7010E94B7
:100A00002D0160E089810E94FD00C7010E942D0137
:100A1000EFEF2E1A3E0A4E0A5E0AE7CF8B810E9444
:100A2000FD00C4010197F1F786E591E000C383352D
:100A300009F0D6C18091C901082E000C990BC0970E
:100A4000789E9001799E300D11240091CA01002EEC
:100A5000000C110B00531109020F131F2091CC0140
:100A6000022E000C330B20533109729EC001739E7D
:100A7000900D11242091CD01022E000C330B205338
:100A80003109A901480F591F5C834B838091DC0118
:100A9000082E000C990BC097789E9001799E300D1E
:100AA00011248091DD01082E000C990BC097F901EB
:100AB000E80FF91FFA83E9838091CF01082E000C1B
:100AC000990BC097689E6001699ED00C112480919B
:100AD000D001082E000C990BC097789E9001799E4A
:100AE000300D11242C0D3D1DC090D1010C2C000C9B
:100AF000DD08C601C0976901C80ED91EA091D301B7
:100B00000A2E000CBB0BD09720E836E948E950E0EC
:100B10000E9449081B012C01A091D4010A2E000C4F
:100B2000BB0BD09720E432E44FE050E00E9449082C
:100B3000260E371E481E591EA091D5010A2E000C04
:100B4000BB0BD09720EA36E841E050E00E9449080C
:100B5000DC01CB01820D931DA41DB51DE091D601D2
:100B60000E2E000CFF0BF09740E157E2E49F90013E
:100B7000E59F300DF49F300D1124A901330F660B52
:100B8000770B840F951FA61FB71FE091D7010E2E7C
:100B9000000CFF0BF09748EE53E0E49F9001E59FB7
:100BA000300DF49F300D1124A901330F660B770B24
:100BB000840F951FA61FB71FE091D8010E2E000CC1
:100BC000FF0BF0976E9E90016F9E300D1124A901CE
:100BD000330F660B770B480F591F6A1F7B1F20913D
:100BE000D901022E000C330B20533109729EC00133
:100BF000739E900D1124092E000CAA0BBB0B480FFD
:100C0000591F6A1F7B1F2091DA01022E000C330B43
:100C100020533109C901330FAA0BBB0B1A012B0159
:100C2000280E391E4A1E5B1E8091C601082E000C3C
:100C3000990BC097789E9001799E300D1124809178
:100C4000C701082E000C990BC097820F931FB82E76
:100C50000E948C00A02E802F0E948C008B810E940D
:100C60008C0071018BEE91E00E9485011816190627
:100C700094F58BEE91E00E948501181619065CF53B
:100C80008BEE91E00E9463019091A5019923F1F010
:100C9000E091A4018E3371F0AE2FB0E0AA55BE4FA3
:100CA0008C93EF5FE093A401ED31A8F05CE15093E9
:100CB000A40111C0F0E0EA55FE4F10821092A50188
:100CC0001092A40181E08093C30105C08C3319F414
:100CD00091E09093A5018091C301882371F0109257
:100CE000C3018091A601843541F484E691E00E941D
:100CF0002F0283E391E00E942F0260E08B810E942B
:100D0000FD0060E0802F0E94FD008601000F111F92
:100D10000C0D1D1D220C331C89810E94D4000197EB
:100D200009F054C060E08A2D0E94FD00CC24C394D9
:100D3000D12C61E0EC14FD048CF08B2D0E94FD00A1
:100D4000C8010E942D0160E08B2D0E94FD00C801AA
:100D50000E942D01EFEFCE1ADE0AEBCF8A2D0E9402
:100D6000FD00CC24C394D12C2C143D0494F061E0FC
:100D70008B2D0E94FD00C8010E942D0160E08B2D8B
:100D80000E94FD00C8010E942D01FFEFCF1ADF0A6B
:100D9000EBCF60E08A2D0E94FD00CC24C394D12CBF
:100DA000EC14FD040CF4B8CF61E08B2D0E94FD0023
:100DB000C8010E942D0160E08B2D0E94FD00C8013A
:100DC0000E942D012FEFC21AD20AEACF61E08B8177
:100DD0000E94FD00C4010197F1F78EE791E027C161
:100DE000883409F022C18091C901082E000C990BAA
:100DF000C097789E9001799E300D11240091CA0110
:100E0000002E000C110B00531109020F131F20912B
:100E1000CC01022E000C330B20533109729EC0010D
:100E2000739E900D1124E090CD010E2C000CFF0854
:100E300040E3E41AF108E80EF91E2091CF01022EDA
:100E4000000C330B20533109729EC001739E900D2C
:100E500011242090D001022C000C330850E3251AF5
:100E60003108280E391E8091D201082E000C990BF2
:100E7000C097689EA001699E500D11248091D301F6
:100E8000082E000C990BC097789E9001799E300D2A
:100E90001124240F351F8091D401082E000C990BCA
:100EA000C097A901480F591F5A834983C090D601A2
:100EB0000C2C000CDD0850E3C51AD108A090D80115
:100EC0000A2C000CBB0880E3A81AB1088091C60167
:100ED000082E000C990BC097789E9001799E300DDA
:100EE00011248091C701082E000C990BC097820F26
:100EF000931F582E0E948C00402E802F0E948C0041
:100F00008E2D0E948C0060E08E2D0E94FD006C2DC5
:100F1000802F91E0A916B10409F043C00E94FD00A2
:100F2000822D0E94D400892B89F461E0852D0E94D6
:100F3000FD0089819A810E942D0160E0852D0E942B
:100F4000FD0089819A810E942D01EACFE1E0CE1651
:100F5000D10411F460E003C0CD2821F461E0802FBA
:100F60000E94FD0008E512E061E0852D0E94FD0071
:100F700089819A810E942D0160E0852D0E94FD00EB
:100F800089819A810E942D010150110969F761E060
:100F90008E2D0E94FD00C4010197F1F782E891E0D7
:100FA00046C00E94FD0001E010E0A016B1067CF3EF
:100FB000822D0E94D400892B89F461E0852D0E9446
:100FC000FD0089819A810E942D0160E0852D0E949B
:100FD000FD0089819A810E942D01EACF842D0E9413
:100FE000D400019749F460E0842D0E94FD0084E85C
:100FF000C82E83E0D82E02C061E0F6CF61E0852DD7
:101000000E94FD0089819A810E942D0160E0852D5A
:101010000E94FD0089819A810E942D01F1E0CF1A82
:10102000D10861F70F5F1F4FC0CF80E991E00E94A8
:101030002F020E9425026ECBEBEEF1E013821282AA
:1010400088EE93E0A0E0B0E084839583A683B78325
:1010500084E091E09183808385EC90E0958784879C
:1010600084EC90E09787868780EC90E0918B808B72
:1010700081EC90E0938B828B82EC90E0958B848B5B
:1010800086EC90E0978B868B118E128E138E148EC9
:101090000895B7FF0C9457080E945708821B930BC2
:1010A0000895EE0FFF1F0590F491E02D09940E9422
:1010B0006208A59F900DB49F900DA49F800D911D77
:1010C00011240895A29FB001B39FC001A39F700D8A
:1010D000811D1124911DB29F700D811D1124911D40
:1010E000089581E090E0F8940C947608F894FFCF8E
:1010F00000000000BC013801850163017701030293
:101100000D0A0033447374756666734E4C20536C3D
:1011100069646572204669726D7761726520563028
:101120002E330057616974696E6720666F722063A1
:101130006F6D6D616E6420746F2070726F63657384
:10114000732E2E2E0A004D6F766520636F6D706CC6
:1011500065746500426F745F436F6E74726F6C20CC
:101160004669726D776172652056302E3200534F9A
:101170004B00486F6D6520706F736974696F6E0006
:10118000556E6B6E6F7720436F6D6D616E642021BD
:0211900021003C
:00000001FF
